:104C84000000090101240200000301FA0400FA05EE
:104C940000020A0A5A0B000F0C00FA0D00030E0062
:104CA400030F0132100096120132130AFA140102A2
:104CB40015010117010A18010A1905321A010A1B04
:104CC400010A1C053223011E2400642A00FA2B0069
:104CD400FA2C50782D003C2E00462F001E30006424
:104CE4003250783300003432FA35016436016437C7
:104CF4000150380A643C00643E003C3F000140FF20
:104D0400FF411450420A5A430AC844053245007808
:104D14004600FA4701224802034C00FA4EFFFF50B6
:104D24000606510596521432530B28540A9656011E
:104D340002570546580001590A465A32FA5B010ADD
:104D44005C14325E000A5F00FE61FFFF64021067BC
:104D540001036A0A3C6B00006C32967801327901D7
:104D640032FAFAFA0000090101240200000301FAF0
:104D74000400FA0500020A0A5A0B000F0C00FA0D8F
:104D840000030E00030F0132100096120132130AC1
:104D9400FA14010215010117010A18010A19053252
:104DA4001A010A1B010A1C053223011E2400642A6D
:104DB40000FA2B00FA2C50782D003C2E00462F00D0
:104DC4001E3000643250783300003432FA35016406
:104DD400360164370150380A643C00643E003C3FAD
:104DE400000140FFFF411450420A5A430AC84405D7
:104DF400324500784600FA4701224802024C00FA84
:104E04004EFFFF500606510596521432530B285498
:104E14000A96560101570546580000590A465A3267
:104E2400FA5B010A5C14325E000A5F00FE61FFFF58
:104E34006402106701036A0A3C6B00006C329678C6
:104E44000132790132FAFAFA0065006F00790083C1
:104E5400008D009700A100AC00B600C000CA00D4C9
:104E640000DE00E800F2005B0063006A0072007A72
:104E7400008200890091009900A100A800B000B848
:104E840000BF00C700CF00D600DF00E600EE00F64A
:104E940000400046004C00520059005F0065006B62
:104EA40000710077007D00830089008F0095009CCD
:104EB40000A200A800AE00B400BA00C000C600CC36
:0C4EC40000D200D900DF00E500EB00F197
:10009E00AE33AF34740A8E048F05FF1200858C3593
:1000AE008D36AE33AF34740A8E048F05FF12515362
:1000BE008C338D34E53445336013740AC39534FFA5
:1000CE00E49533FE8E338F34783512519FE550A868
:1000DE0035B80015D395364010E550C39536FFE47C
:1000EE009535FE8E358F368010E5502424C3953617
:1000FE00FFE49535FE8E358F36755000AE35AF3632
:10010E00740B6F4E6006740C6F4E7018AE35AF36B2
:10011E00740B6F4E70057550018003755002753665
:10012E000A753500AE35AF3674176F4E600674180B
:10013E006F4E7018AE35AF3674176F4E7005755022
:10014E00018003755002753616753500AE35AF3623
:10015E0074236F4E600674246F4E7018AE35AF3632
:10016E0074236F4E700575500180037550027536FD
:10017E002275350022900085E0B40104C20C800285
:10018E00D20C900086E0B40104C20D8002D20D9014
:10019E0000C3E075F0DCA4FFAEF0740A8E048F0588
:1001AE00FF1200859007ABECF0A3EDF0A20740160E
:1001BE0074038C068D07125138740112512A900760
:1001CE00A9EEF0A3EFF07E017F00900081E01251C6
:1001DE00389000C4E08E048F05FF120085740AFF6C
:1001EE001200858D399000CDE075F0DCA4FFAEF0E5
:1001FE00740A8E048F05FF1200859007AFECF0A3F2
:10020E00EDF09000CFE060139000CFE0F5F07416A3
:10021E0084FF7E00EF9007B7F0800674649007B7F6
:10022E00F09000D7E0B4020674029000B9F090008E
:10023E00AEE0B40B0874E390006FF080499000AE0E
:10024E00E0B419129000C4E0904E3712511BE493A3
:10025E0090006FF080309000AEE0B41E129000C49B
:10026E00E0904E5512511BE49390006FF080179062
:10027E0000AEE0B428109000C4E0904E7F12511BE7
:10028E00E49390006FF09000E1E0B4011790002429
:10029E00740FF0A374FFF0900026E4F0A3F0740244
:1002AE009000E1F09000E1E0B40341900026E0FE02
:1002BE00A3E0FF900024E0FCA3E0FD125197741020
:1002CE00125138740812512AEF90006CF0EF70063C
:1002DE0074FF90006CF074009000E1F0900025E047
:1002EE0090006DF0900024E090006EF0900072E0AF
:1002FE00900034F0900034E0240C900035F0900023
:10030E0034E02418900036F0900035E0D394244069
:10031E000B900035E0C39424900035F0900036E049
:10032E00D39424400B900036E0C39424900036F012
:10033E0090003AE4F0900034E0640B6007900034D3
:10034E00E0B40C20900034E0B40B06740290003A36
:10035E00F0900034E0B40C0690003A7401F0740D85
:10036E00900034F0900034E064176007900034E0A1
:10037E00B41820900034E0B41706740290003AF0DE
:10038E00900034E0B4180690003A7401F07419909D
:10039E000034F0900034E064236007900034E0B441
:1003AE002420900034E0B42306740290003AF090BA
:1003BE000034E0B4240690003A7401F090003474D6
:1003CE0001F090003BE4F0900035E0640B60079084
:1003DE000035E0B40C20900035E0B40B06740290AA
:1003EE00003BF0900035E0B40C0690003B7401F039
:1003FE00740D900035F0900035E0641760079000A2
:10040E0035E0B41820900035E0B417067402900061
:10041E003BF0900035E0B4180690003B7401F07488
:10042E0019900035F0900035E06423600790003598
:10043E00E0B42420900035E0B42306740290003B13
:10044E00F0900035E0B4240690003B7401F090006B
:10045E00357401F090003CE4F0900036E0640B60DF
:10046E0007900036E0B40C20900036E0B40B067412
:10047E000290003CF0900036E0B40C0690003C7404
:10048E0001F0740D900036F0900036E064176007AE
:10049E00900036E0B41820900036E0B417067402CF
:1004AE0090003CF0900036E0B4180690003C7401C9
:1004BE00F07419900036F0900036E06423600790D7
:1004CE000036E0B42420900036E0B4230674029087
:1004DE00003CF0900036E0B4240690003C7401F02D
:1004EE009000367401F0900072E0FE9000D5E02E80
:1004FE0090003EF090003EE0D39424400B90003EDE
:10050E00E0C3942490003EF090003EE0B4120674D6
:10051E001390003EF090003EE0B4240690003E742E
:10052E0001F090003EE0640B600F90003EE0641717
:10053E00600790003EE0B4230690003EE014F09079
:10054E00003EE0640C600790003EE0B41706900099
:10055E003EE004F090003EE0D39412400D90003E39
:10056E00E0C3941290003FF0800A90003EE0241207
:10057E0090003FF09000B8E0900037F0900037E028
:10058E00640B6007900037E0B41706900037E01454
:10059E00F0900037E0640C6007900037E0B4180666
:1005AE00900037E004F0900037E0240C900038F013
:1005BE00900037E02418900039F0900038E0D39482
:1005CE0024400B900038E0C39424900038F0900043
:1005DE0039E0D39424400B900039E0C3942490006A
:1005EE0039F022C293C294C291C292C287C290E5E0
:1005FE00B554EFF5B5E5B554DFF5B5C296C295C263
:10060E00A0C297C2A2C2A1E5B5547FF5B5E5B55417
:10061E00BFF5B5E5B554FBF5B5C20E75374690007E
:10062E00BBE07005754902800375490390000C7498
:10063E00FFF0A374DCF090009CE0900012F8E4F060
:10064E00E8A3F0C214C216C21874C8900028F07441
:10065E00C890002CF074C8900030F07526007525F7
:10066E0000C207756D00E54BB40903754B00753C70
:10067E000090001AE4F0A3F0754C1E752800752743
:10068E0000C211C212C2139007ABE0FEA3E0FF74CA
:10069E0003125138740112512A9007A9EEF0A3EFFC
:1006AE00F0C203900010E4F0A3F0C21F755200C216
:1006BE0009C208C21C900070E4F022053D2285A7F5
:1006CE004F75A7109000B9E0640360079000D7E063
:1006DE00B4022CA2D8B34002C293A2D9B34002C234
:1006EE0094A2DAB34002C291A2DBB34002C292A23C
:1006FE00DCB34002C287A2DDB34002C290801BA2CF
:10070E00D8B34004C293C292A2D9B34004C294C2D9
:10071E0087A2DAB34004C291C29075D840854FA724
:10072E0022900047E4936406600280FE74C890072E
:10073E00B1F8E4F0E8A3F075B50075840175A70073
:10074E0075FF8075EF0690003DE4F075C91075A732
:10075E000F75A1C775A70075D90075CE0C75A70FBB
:10076E0075F1FE75F2FF75F30775F47875A4BA7519
:10077E00A5FF75A60775AE0075AFFF75D48175D54B
:10078E00FF75D6FF75D7FF75A70075A20175A14736
:10079E0075F80975D80075D90475A71075D8007548
:1007AE00D90475DA0975DB0975DC0975DD0975DEA5
:1007BE000975DF0975D84075A70075E60075E71055
:1007CE0075BC0175BE0475BD6C75BE0775BDA07593
:1007DE00BE0875BD0175BC0075BB1875BC2075BA19
:1007EE000875E88075D11375B50075A70F75E1050D
:1007FE0075E20075C740C293C294C291C292C2877D
:10080E00C290E5B554EFF5B5E5B554DFF5B5C29632
:10081E00C295C2A0C297C2A2C2A1E5B5547FF5B5DA
:10082E00E5B554BFF5B5E5B554FBF5B5759700754F
:10083E009780740A1200757597C0E5975420700260
:10084E0080F8758F0275A700D2AF75980075A90C48
:10085E0075A70F75AB4375ADFB75AC1E75A71075FF
:10086E00C91875CA0075CB0075C80475A7007589BF
:10087E0012758E04758C00758A00C2A9D28C758D86
:10088E0000758B00D2ABD28E75D94475320075319E
:10089E0000752E00752D00754600754700C29974BF
:1008AE00C8F5097508001230DA75B5007463900743
:1008BE00B1F8E4F0E8A3F01233667464F509750834
:1008CE00001230DAC21E90005AE0B40108A2B54000
:1008DE0002D21E802E90005AE0B4021175A70F7539
:1008EE00F30F75A700A2A34002D21E801690005AE5
:1008FE00E0B4030F75A70F75F31775A700A2A440F8
:10090E0002D21EA21EB350030209FF74089007B153
:10091E00F8E4F0E8A3F01232357464F509750800B6
:10092E001230DA74099007B1F8E4F0E8A3F012324D
:10093E00357464F5097508001230DA740A9007B13F
:10094E00F8E4F0E8A3F01232357464F50975080086
:10095E001230DA740B9007B1F8E4F0E8A3F012321B
:10096E00357464F5097508001230DA740C9007B10D
:10097E00F8E4F0E8A3F01232357464F50975080056
:10098E001230DA740D9007B1F8E4F0E8A3F01232E9
:10099E00357464F5097508001230DA740E9007B1DB
:1009AE00F8E4F0E8A3F01232357464F50975080026
:1009BE001230DA74029000BAF090005AE090007E85
:1009CE00F090005AE0B401087400900086F0801C8C
:1009DE0090005AE0B4020874009000C9F0800D90A7
:1009EE00005AE0B4030674009000D6F0D21B020A3F
:1009FE00DF9007B1E4F0A304F01232357464F50908
:100A0E007508001230DA74029007B1F8E4F0E8A32A
:100A1E00F01232357464F5097508001230DA740379
:100A2E009007B1F8E4F0E8A3F01232357464F509DA
:100A3E007508001230DA74049007B1F8E4F0E8A3F8
:100A4E00F01232357464F5097508001230DA740547
:100A5E009007B1F8E4F0E8A3F01232357464F509AA
:100A6E007508001230DA74069007B1F8E4F0E8A3C6
:100A7E00F01232357464F5097508001230DA740715
:100A8E009007B1F8E4F0E8A3F01232357464F5097A
:100A9E007508001230DA74019000BAF090005AE036
:100AAE0090007EF090005AE0B40108740090008629
:100ABE00F0801C90005AE0B4020874009000C9F057
:100ACE00800D90005AE0B4030674009000D6F0C278
:100ADE001B1234DA9000C4E07006740A9000C4F061
:100AEE0090006FE0700674E390006FF0120183E5E2
:100AFE00B54401F5B57406900049F0740190004AB2
:100B0E00F0740390004CF0740490004DF0742A9031
:100B1E00004EF0740590004FF090004BE0B40406C8
:100B2E00740490004FF07403900050F07400900025
:100B3E0055F07400900056F07401900057F0740058
:100B4E00900058F074FF900059F07433900148F003
:100B5E007436900149F0742D90014AF0743690016C
:100B6E004BF0742090014CF0744E90014DF074696E
:100B7E0090014EF0747390014FF07473900150F029
:100B8E007461900151F0746E900152F074339001C3
:100B9E0053F07435900154F07430900155F0745A3E
:100BAE00900156F09000E0E090006CF0900097E01D
:100BBE0090006DF0900098E090006EF0C214C21696
:100BCE00C21874C8900028F074C890002CF074C835
:100BDE00900030F0C211C212C213755200C209C287
:100BEE0008C21C900070E4F0A2B6B3920AA2B3B38E
:100BFE00920B752600752500753746754C1E9000B4
:100C0E0068E4F075271975286490000C74FFF0A342
:100C1E0074DCF0C20E754B00C207752A00752900F0
:100C2E00900010E4F0A3F0743A900771F074FD9008
:100C3E000772F0756E00900069E4F0752C00752B4C
:100C4E0000900014E4F0A3F090009CE0900012F8E5
:100C5E00E4F0E8A3F090007DE075F032A4FFAEF072
:100C6E00900022EEF0A3EFF09007ABE0FEA3E0FFC2
:100C7E007403125138740112512A9007A9EEF0A391
:100C8E00EFF0754A0174FA900045F0C21F756D00C1
:100C9E00753C00C20FC210C220C203754D00C204C3
:100CAE00D205C206D21D74FE900040F074FE900074
:100CBE0041F0753800754400753A00753E32753F47
:100CCE0000754000743C900043F0743C900044F07A
:100CDE0075410075420075430090001AE4F0A3F0D0
:100CEE00754500D2B2D2A4D2B0D2B1D2A3D2A7D27D
:100CFE00A6D2A5D2B790007DE0D394FA400674FA3E
:100D0E0090007DF07E017F0090006EE012513890D1
:100D1E00006DE02FFF50010E900024EEF0A3EFF0D7
:100D2E00EFD394FFEE940F4007900024E4F0A3F06D
:100D3E0090006CE0700674FF90006CF09000BAE0CA
:100D4E00D39402400674019000BAF09000BBE0709C
:100D5E000575490280037549039000BCE0D39401E8
:100D6E00400674009000BCF09000C2E0C3940A509C
:100D7E0006740A9000C2F09000CCE07006740190E8
:100D8E0000CCF09000CCE0B4FF0674FE9000CCF0E6
:100D9E009000D3E0D394FE400674FE9000D3F0741E
:100DAE00019000D9F074019000DAF074009000DC2C
:100DBE00F074009000E1F0D29CD2EC75CF01A298B5
:100DCE00B350030211BFC298E54764046006E5996B
:100DDE0064FF6002801EE547600874E625479000B8
:100DEE0045F0754700E546600874F02546900045CD
:100DFE00F0754600E5476003020EA4754700E599BD
:100E0E00B4FF03754601E599B4FE03754602E599F4
:100E1E00B4FD03754603E599B4FC03754604E599E4
:100E2E00B4FA03754605E599B4FB03754701E599D8
:100E3E00B4F903754704E599D394E54007E599C3E2
:100E4E0094F0400280168599487547027E017F0016
:100E5E00E548C394E61251388E2F8F3075320075E7
:100E6E003100E599D394C74007E599C394E6400253
:100E7E00801F85994875470374E5C39548F530750D
:100E8E002F00AE2FAF30904ED01200647831125139
:100E9E007DD2990211BFE547B401028003020F8291
:100EAE00E532453170031205F1AE31AF329000716B
:100EBE0012515FE599F0783112519FAE31AF32EF9A
:100ECE00B40106EEB407028003020F82900771E0B0
:100EDE00B43C028003020F6CC29C12018390006C22
:100EEE00E09000E0F090006DE0900097F090006EC2
:100EFE00E0900098F0A21B4032755001E550D3945B
:100F0E00075026E5509007B1F8E4F0E8A3F074AA74
:100F1E0090003DF01231067464F509750800123028
:100F2E00DA7850740126F650D38030755008E550AB
:100F3E00D3940E5026E5509007B1F8E4F0E8A3F0F4
:100F4E0074AA90003DF01231067464F5097508001C
:100F5E001230DA7850740126F650D31234DA74C88F
:100F6E009007B1F8E4F0E8A3F0D29C7547007546FF
:100F7E00007599FBE547B402028003021016E532B4
:100F8E004531700685992E752D00AE31AF32740144
:100F9E006F4E701BAC2DAD2EAA2FAB30ED2BFBEC94
:100FAE003AFA8A068B0790007112515FE599F07834
:100FBE003112519FAE31AF3274026F4E704AAC2D6A
:100FCE00AD2E740D6D4C702774639007B1F8E4F07C
:100FDE00E8A3F074AB90003DF090007EE090005AD4
:100FEE00F012343F74C89007B1F8E4F0E8A3F0AE05
:100FFE002DAF2E74566F4E70031205F112018385BC
:10100E004899754700754600E547B4033FAE31AFCA
:10101E003290007112515FE599F0783112519FAE06
:10102E0031AF32AC2FAD308F028E038C068D079010
:10103E004F0C120064E493F9740193FEEAD39EEB15
:10104E00994009854899754700754600E547B404EF
:10105E000280030211BFE532453170031205F1AE75
:10106E0031AF3290007112515FE599F07831125123
:10107E009FAE31AF32EFB40006EEB4010280030230
:10108E0011BF900053E075F002A4FDACF08D50ED51
:10109E00900071125174EDFAE0FBEA900074125157
:1010AE0074EBFAE0FBEA2BFA900053E0B5020280F3
:1010BE00030211B00DED900071125174E550FDE078
:1010CE00FAED900075125174EAFDE0FAEDC39AFD47
:1010DE00900053E0B5050280030211B0E550900078
:1010EE0073125174E550FDE0FAED900076125174D2
:1010FE00EAFDE0FAED2AFD900053E0B5050280030B
:10110E000211B0E550900077125174FDE0FAED90A7
:10111E000053E0F4042A90005AF0E5509000781243
:10112E005174FDE0FAED900053E0F4042A90005B58
:10113E00F0E550900079125174FDE0FAED900053F5
:10114E00E0F4042A90005CF0E55090007A1251749D
:10115E00FDE0FAED900053E0F4042A9007B1F8E4B4
:10116E00F0E8A3F074AB90003DF012343F7464F5D8
:10117E00097508001230DA9007B112514612343F49
:10118E007464F5097508001230DA9007B1125146F1
:10119E0012343F7599F97464F5097508001230DA46
:1011AE0080FE7599FF7464F5097508001230DA80B7
:1011BE00FEE5466006A299B3B3400302133DC29901
:1011CE00E546B4011FAE31AF3290004912515FE0D7
:1011DE00F599783112519FAE31AF3274116F4E7056
:1011EE0003754600E546B40203854A99E546B40305
:1011FE001DAE31AF3290007112515FE0F599EFB430
:10120E000107EEB40703754600783112519FE5468B
:10121E00B4040280030212FFE532453170038526C5
:10122E0099AE31AF3274016F4E7003853899AE317D
:10123E00AF3274026F4E7003853A99AE31AF32748D
:10124E00036F4E7003853E99AE31AF3274046F4E0C
:10125E007003854099AE31AF3274056F4E700385C1
:10126E004199AE31AF3274066F4E7003854299AE1E
:10127E0031AF3274076F4E7003854399AE31AF3282
:10128E0074086F4E700690001BE0F599AE31AF32C8
:10129E0074096F4E7006900045E0F599AE31AF328D
:1012AE00740A6F4E7003854499AE31AF32740B6F72
:1012BE004E7003853F99AE31AF32740C6F4E700392
:1012CE00854599AE31AF32740D6F4E700590004565
:1012DE00E4F0AE31AF32740D6F4E70037599FC7839
:1012EE003112519FAE31AF32740E6F4E7003754690
:1012FE0000E546B4053990004BE0D394044010AE9F
:10130E0031AF32904C8412515FE493F599800EAE5A
:10131E0031AF32904D6812515FE493F599AE31AF13
:10132E003274E36F4E7003754600783112519FE5AB
:10133E004764016005E547B40403020DC9C28E7E01
:10134E00107F00E53D125138E58D75F010A4FDAC0F
:10135E00F0EF2DFDEE3CFCE58B75F01084FF7E006A
:10136E00ED2FFFEC3EFE8E278F28D28E90009EE052
:10137E00605690001C12514690001CE0FCA3E0FD4C
:10138E0090001EE0FAA3E0FBEDB5033CECB502388D
:10139E00B21AA207B34013A21AB34008E5B544042B
:1013AE00F5B58006E5B554FBF5B590001EE0FEA33D
:1013BE00E0FF900020E0FCA3E0FDEF2DFDEE3CFCF5
:1013CE0090001EECF0A3EDF09000ABE060099000F1
:1013DE00ABE0C3940340030214691249DAA207B3C7
:1013EE005009900068E0C394284002800690009552
:1013FE00E0F56CE56C75F005A4FFAEF09007B3EE6A
:10140E00F0A3EFF0900082E0C3953A4007E538C3B1
:10141E00953950079007B3E4F0A3F0AE59AF5A9048
:10142E0007B3E0FCA3E0FDEFD39DEE9C4004C2A108
:10143E00800B900068E0C3943C5002D2A19000ABA8
:10144E00E0B402109000B9E0C3940350079000D7A7
:10145E00E0B401028005A2A1B392A29000ABE0B469
:10146E00031C124AD6AE59AF5A9007B3E0FCA3E064
:10147E00FDEFD39DEE9C4004D2A18002C2A190004C
:10148E0086E06009A2B3300B01B3B34002805BA2C9
:10149E00B3300B01B34053A2B3300D01B34018A2C9
:1014AE000DB3920B900070E0D3941240057552016B
:1014BE00D208900070E4F0A20DB330B301B3402A0D
:1014CE00E552B40112900070E0D3940740099000E9
:1014DE0070E0C3940C40028005755202D209E552A9
:1014EE00B40103755200A20D920BA2B6300A01B3DD
:1014FE005003021A98A2B6300A01B35003021A988A
:10150E00A2B6300C01B350030219D0754A009000F8
:10151E0070E004F090009EE07013A20CB34008E55A
:10152E00B554FBF5B58006E5B54404F5B50537A20F
:10153E000EB3B35013AE27AF2890000CE0FCA3E01F
:10154E00FDEDC39FEC9E4003021659E537B40B0622
:10155E0075370D021631E537B417067537190216B1
:10156E0031E549B40330E537B42305754901801FD1
:10157E00A21FB3401AE537C394235006900045745A
:10158E0001F0E537D3942340067402900045F075C0
:10159E003701D21F8044E549B402067549017537FB
:1015AE0023E537B42305753701802F900045E07091
:1015BE001AE537C3942350069000457401F0E537C1
:1015CE00D3942340067402900045F09000BBE0B423
:1015DE0002051205F1800375370190009EE060430D
:1015EE0090001CE0FEA3E0FF90009EE08E048F05AD
:1015FE00FF12008574018C068D0712512A9000206F
:10160E00EEF0A3EFF0900020E0F8A3E090001EC8EB
:10161E00F0A3C8F090001CE4F0A3F0C21AE5B55494
:10162E00FBF5B5E552B40206753701755200AE29C9
:10163E00AF2AAC27AD28EF2DFDEE3CFC74028C06D4
:10164E008D0712512A8E298F2A802BAE29AF2AACF4
:10165E0027AD28EF2DFDEE3CFC74018C068D071294
:10166E00512A8E298F2AAC27AD28EDD39488EC947D
:10167E001340031205F1E537B423107403900045AF
:10168E00F09000BBE0B402031205F1AE2BAF2CAC10
:10169E0027AD28EF2DFDEE3CFC8C2B8D2CAE27AF0D
:1016AE0028EFD39DEE9C4011900014E0FAA3E0FBCE
:1016BE00EBC394E8EA9403400280069000141251A2
:1016CE0046900010E0FEA3E0FFAC27AD28EF2DFD05
:1016DE00EE3CFC900010ECF0A3EDF09000BBE0B4FB
:1016EE000218AE27AF287405125138740112512A10
:1016FE0090000CEEF0A3EFF08011AE27AF2874022D
:10170E0012513890000CEEF0A3EFF0C28E758D00E2
:10171E00758B00753D00752801752700D28EE53753
:10172E00240875F00984AFF07E00EF4E70759000BE
:10173E0010E0F8A3E090000EC8F0A3C8F090000EE1
:10174E00E0FEA3E0FFEF4E600B7C807D0E12503A60
:10175E008E258F26900010E4F0A3F0AE25AF2674F0
:10176E0028BE00039F5010E53C2FFF50010E740160
:10177E0012512A8E258F2685263C9000C2E0A82580
:10178E00B8000DD395264008E526900042F080095A
:10179E009000C2E014900042F0E549600675260004
:1017AE007525009000B9E0B40308900037E0653766
:1017BE0060028026A209B34004D21C8002B21C90A3
:1017CE000086E0600BA209B35006A21CB3B3400220
:1017DE0080067404900045F0C209E537640A60057E
:1017EE00E537B418099000ABE0600312471C900077
:1017FE00B0E0701490003EE06537600790003FE067
:10180E00B53703754B00801E90003EE065376013C0
:10181E0090003EE0240C6537600990003EE02418ED
:10182E00B53703754B00A20F5003021925900077B0
:10183E00E0B4015AE54075F00584FF7E0090057115
:10184E0012515FE0F534753300AE33AF349000754E
:10185E00E012513874648E048F05FF12008574C136
:10186E008C068D071251388E358F36900012E0FEA1
:10187E00A3E0FFAC33AD3412000374648E048F0505
:10188E00FF120085900012ECF0A3EDF0800F900097
:10189E0075E075F0C1A4FFAEF08E358F36E53AC314
:1018AE0094CC507175A71085F95085FA517E017F41
:1018BE0000E551125138E5502FFF50010E8E338F37
:1018CE0034AC35AD36EF2DFDEE3CFC8C358D36D27D
:1018DE0093D294D291E536F5FBE535F5FCE536F578
:1018EE00E9E535F5EAE536F5EBE535F5EC9000B9C9
:1018FE00E0B4031ED292D287D290E536F5EDE535EF
:10190E00F5EEE536F5FDE535F5FEE536F5CEE535D4
:10191E00F5CF75A700D20FE549B40106A208B3B3FF
:10192E004002800F754C019000487401F0E5B544FB
:10193E0001F5B5E54960030219CB9000BEE0600DDC
:10194E009000C5E0A825B8000695264002803A9082
:10195E0000BEE0B4021F900034E06537600F9000C7
:10196E0035E065376007900036E0B53703754C03F8
:10197E00754500800CC20075450090001AE4F0A376
:10198E00F07409900045F08034900034E0B5370BC8
:10199E00754C019000487401F08022900035E0B53E
:1019AE00370B754C017402900048F0801090003691
:1019BE00E0B53709754C017403900048F0A20CB3E2
:1019CE00920AA20CB330B601B35003021A98754AAC
:1019DE000190009EE07013A20CB34008E5B54404DC
:1019EE00F5B58006E5B554FBF5B5A20C920AE537C0
:1019FE00D3944A4012D20EE537D39469400974034A
:101A0E00900045F07537469000C6E0B40107E543F7
:101A1E00C39414400280031205F17428900068F0FC
:101A2E00A204300501B35017A204B34008E5B54433
:101A3E0008F5B58006E5B554F7F5B5A2049205E5AF
:101A4E0043C394415009740E900045F01205F19075
:101A5E00004FE0FE90004BE004C39E400990004B07
:101A6E00E0D39406400974FB900045F01205F19006
:101A7E000054E06015900054E0FE90004EE06E6061
:101A8E000974FE900045F01205F1A211B3B350088F
:101A9E00900037E065376003021B86A202B3500642
:101AAE00A200B3B34003021B8075A71085F95085C1
:101ABE00FA517E017F00E551125138E5502FFF504B
:101ACE00010E8E338F34900018E0FCA3E0FDEF2D55
:101ADE00FDEE3CFC8C358D369000B9E0B4034EA281
:101AEE0007B34028A21CB3400CE536F5FBE535F5EF
:101AFE00FCD293800AE536F5EDE535F5EED292A2ED
:101B0E0003B34004D2A28002C2A2801FE536F5FBC9
:101B1E00E535F5FCE536F5EDE535F5EED293D292E9
:101B2E00A203B34004D2A28002C2A280429000D788
:101B3E00E0C394025013E536F5FBE535F5FCD29380
:101B4E00A203B34002D2928026E536F5FBE535F5C9
:101B5E00FCD293AE33AF34AC57AD58EF2DFDEE3C07
:101B6E00FC8C358D36E536F5EDE535F5EED2927514
:101B7E00A700C211D212D213A212B3B35008900012
:101B8E0038E065376003021C74A202B35006A2004F
:101B9E00B3B34003021C6E75A71085F95085FA5138
:101BAE007E017F00E551125138E5502FFF50010E96
:101BBE008E338F34900018E0FCA3E0FDEF2DFDEE88
:101BCE003CFC8C358D369000B9E0B4034EA207B3C1
:101BDE004028A21CB3400CE536F5E9E535F5EAD20E
:101BEE0094800AE536F5FDE535F5FED287A203B3FE
:101BFE004004D2A28002C2A2801FE536F5E9E53587
:101C0E00F5EAE536F5FDE535F5FED294D287A20369
:101C1E00B34004D2A28002C2A280429000D7E0C399
:101C2E0094025013E536F5E9E535F5EAD294A203B0
:101C3E00B34002D2878026E536F5E9E535F5EAD2DE
:101C4E0094AE33AF34AC57AD58EF2DFDEE3CFC8C5B
:101C5E00358D36E536F5FDE535F5FED28775A700EF
:101C6E00D211C212D213A213B3B35008900039E0AE
:101C7E0065376003021D62A202B35006A200B3B321
:101C8E004003021D5C75A71085F95085FA517E013F
:101C9E007F00E551125138E5502FFF50010E8E3363
:101CAE008F34900018E0FCA3E0FDEF2DFDEE3CFC20
:101CBE008C358D369000B9E0B4034EA207B34028A0
:101CCE00A21CB3400CE536F5EBE535F5ECD2918070
:101CDE000AE536F5CEE535F5CFD290A203B3400432
:101CEE00D2A28002C2A2801FE536F5EBE535F5ECF7
:101CFE00E536F5CEE535F5CFD291D290A203B340BD
:101D0E0004D2A28002C2A280429000D7E0C3940205
:101D1E005013E536F5EBE535F5ECD291A203B34061
:101D2E0002D2908026E536F5EBE535F5ECD291AE94
:101D3E0033AF34AC57AD58EF2DFDEE3CFC8C358DEA
:101D4E0036E536F5CEE535F5CFD29075A700D21132
:101D5E00D212C213E54CB4081812404BA211B35064
:101D6E0005A212B340028006D211D212D213754CC4
:101D7E001EE54CB40706123E03754C08E54CB4063E
:101D8E003D900012E0FEA3E0FFEF4E6006A207B307
:101D9E00B340028023AE53AF54900012E0FCA3E098
:101DAE00FDEF2DFDEE3CFC8C538D54E537D3940C9A
:101DBE005006900012120039123BD5754C07E54CB7
:101DCE00B40506123A35754C06E54CB40432900053
:101DDE00ACE09030BCF82828731236C98012123647
:101DEE00C9800D12387780081239298003123929DB
:0F30BC00021DE7021DEC021DF1021DF6021DFBB5
:101DFE0090008EE060051248058002C204754C0505
:101E0E00E54CB403028003021EEE1248F59000ACBE
:101E1E00E0D39402403F900080E02403A825B80050
:101E2E000495265009900082E0D3953A500280081E
:101E3E00D2027408900045F0900080E0A825B8000A
:101E4E0005D39526500B900082E02403C3953A509B
:101E5E0002C2028039900080E02403A825B8000455
:101E6E0095265007E538C3953940028008D2027492
:101E7E0008900045F0900080E0A825B80005D395A5
:101E8E00265009E539240FC395385002C20290003E
:101E9E00C6E07007E543C3941440028002D202A24A
:101EAE00024005754C04800A754C1E90001AE4F031
:101EBE00A3F0A207B34029E54075F00584FF7E002C
:101ECE0090057112515FE0C394695005124751801D
:101EDE000F9007ABE0F8A3E09007A9C8F0A3C8F0F5
:101EEE00E54CB40A028003021FB090002AE0C394AE
:101EFE00465008C296744690002AF090003AE0B41C
:101F0E00011DE55B240AF55B9007ADE0FEA3E0FF43
:101F1E00740A2FFF50010E9007ADEEF0A3EFF09074
:101F2E00003AE0B4021DE55B2414F55B9007ADE0CA
:101F3E00FEA3E0FF74142FFF50010E9007ADEEF0DC
:101F4E00A3EFF0855B34753300900034E0F550124A
:101F5E00009EE53690002AF0900006E533F0A3E5EA
:101F6E0034F0E55090002BF0C2159007ADE0F5333C
:101F7E00A3E0F534900034E0F55012009EE5369063
:101F8E000028F0900000E533F0A3E534F0E5509022
:101F9E000029F0C214E549B40105754C0B80037598
:101FAE004C03900028E0B53702800302204FA214A4
:101FBE004072900000E0FEA3E0FFEF4E6021AE29DC
:101FCE00AF2A900000E0FCA3E0FD120003740A8E1D
:101FDE00048F05FF120085900000ECF0A3EDF09049
:101FEE000029E0601A900000E0FEA3E0FFAC29ADEE
:101FFE002AEF2DFDEE3CFC900000ECF0A3EDF090EE
:10200E000029E0D39401401A900000E0FEA3E0FF07
:10201E00AC29AD2AEF2DFDEE3CFC900000ECF0A3B8
:10202E00EDF0D214AE27AF28900000E0FCA3E0FD47
:10203E00EFC39DEE9C400AD296C21474C89000283D
:10204E00F0A214B3B35007900028E0B53702800A0F
:10205E00D29674C8900028F0C21490002AE0B537CA
:10206E00028003022107A2154072900006E0FEA333
:10207E00E0FFEF4E6021AE29AF2A900006E0FCA3F0
:10208E00E0FD120003740A8E048F05FF1200859086
:10209E000006ECF0A3EDF090002BE0601A90000625
:1020AE00E0FEA3E0FFAC29AD2AEF2DFDEE3CFC9047
:1020BE000006ECF0A3EDF090002BE0D39401401A53
:1020CE00900006E0FEA3E0FFAC29AD2AEF2DFDEE59
:1020DE003CFC900006ECF0A3EDF0D215AE27AF2835
:1020EE00900006E0FCA3E0FDEFC39DEE9C400AC20B
:1020FE0096744690002AF0C215A215B3B3500790FD
:10210E00002AE0B53702800AC296744690002AF083
:10211E00C215E54CB40B0280030221ED90002EE0B7
:10212E00C3944650139000C7E0B40104C2968002D7
:10213E00C295744690002EF090003BE0B4011DE570
:10214E005B240AF55B9007ADE0FEA3E0FF740A2F57
:10215E00FF50010E9007ADEEF0A3EFF090003BE0C4
:10216E00B4021DE55B2414F55B9007ADE0FEA3E021
:10217E00FF74142FFF50010E9007ADEEF0A3EFF099
:10218E00855B34753300900035E0F55012009EE506
:10219E003690002EF0900008E533F0A3E534F0E51C
:1021AE005090002FF0C2179007ADE0F533A3E0F585
:1021BE0034900035E0F55012009EE53690002CF07C
:1021CE00900002E533F0A3E534F0E55090002DF0D9
:1021DE00C216E549B40105754C0C8003754C03908D
:1021EE00002CE0B537028003022297A216407290AF
:1021FE000002E0FEA3E0FFEF4E6021AE29AF2A9071
:10220E000002E0FCA3E0FD120003740A8E048F05A9
:10221E00FF120085900002ECF0A3EDF090002DE08F
:10222E00601A900002E0FEA3E0FFAC29AD2AEF2D6C
:10223E00FDEE3CFC900002ECF0A3EDF090002DE0E2
:10224E00D39401401A900002E0FEA3E0FFAC29AD4A
:10225E002AEF2DFDEE3CFC900002ECF0A3EDF0D247
:10226E0016AE27AF28900002E0FCA3E0FDEFC39D61
:10227E00EE9C40159000C7E0B40104D2968002D2C5
:10228E0095C21674C890002CF0A216B3B3500790E6
:10229E00002CE0B5370280159000C7E0B40104D2DF
:1022AE00968002D29574C890002CF0C21690002E23
:1022BE00E0B537028003022365A217407290000832
:1022CE00E0FEA3E0FFEF4E6021AE29AF2A9000089A
:1022DE00E0FCA3E0FD120003740A8E048F05FF12CA
:1022EE000085900008ECF0A3EDF090002FE0601A4E
:1022FE00900008E0FEA3E0FFAC29AD2AEF2DFDEE25
:10230E003CFC900008ECF0A3EDF090002FE0D3948D
:10231E0001401A900008E0FEA3E0FFAC29AD2AEFC1
:10232E002DFDEE3CFC900008ECF0A3EDF0D217AEC4
:10233E0027AF28900008E0FCA3E0FDEFC39DEE9CC4
:10234E0040159000C7E0B40104C2968002C2957495
:10235E004690002EF0C217A217B3B3500790002E6E
:10236E00E0B5370280159000C7E0B40104C2968034
:10237E0002C295744690002EF0C217E54CB40C02C2
:10238E008003022466900032E0C3944650139000FE
:10239E00C7E0B40104C2968002C2A0744690003217
:1023AE00F090003CE0B4011DE55B240AF55B90075C
:1023BE00ADE0FEA3E0FF740A2FFF50010E9007ADB3
:1023CE00EEF0A3EFF090003CE0B4021DE55B2414A8
:1023DE00F55B9007ADE0FEA3E0FF74142FFF5001F4
:1023EE000E9007ADEEF0A3EFF0855B3475330090E1
:1023FE000036E0F55012009EE536900032F0900067
:10240E000AE533F0A3E534F0E550900033F0C2193D
:10241E009007ADE0F533A3E0F534900036E0F550CB
:10242E0012009EE536900030F0900004E533F0A3E4
:10243E00E534F0E550900031F0C218E549B40115CD
:10244E0075490074C8900028F074C890002CF07480
:10245E00C8900030F0754C03900030E0B537028024
:10246E0003022510A2184072900004E0FEA3E0FFC4
:10247E00EF4E6021AE29AF2A900004E0FCA3E0FDF0
:10248E00120003740A8E048F05FF1200859000045B
:10249E00ECF0A3EDF0900031E0601A900004E0FE45
:1024AE00A3E0FFAC29AD2AEF2DFDEE3CFC9000041D
:1024BE00ECF0A3EDF0900031E0D39401401A9000BF
:1024CE0004E0FEA3E0FFAC29AD2AEF2DFDEE3CFCAF
:1024DE00900004ECF0A3EDF0D218AE27AF289000D8
:1024EE0004E0FCA3E0FDEFC39DEE9C40159000C7F9
:1024FE00E0B40104D2968002D2A0C21874C8900033
:10250E0030F0A218B3B35007900030E0B537028018
:10251E00159000C7E0B40104D2968002D2A074C810
:10252E00900030F0C218900032E0B53702800302FE
:10253E0025DEA219407290000AE0FEA3E0FFEF4EE6
:10254E006021AE29AF2A90000AE0FCA3E0FD120044
:10255E0003740A8E048F05FF12008590000AECF0BA
:10256E00A3EDF0900033E0601A90000AE0FEA3E0C5
:10257E00FFAC29AD2AEF2DFDEE3CFC90000AECF0ED
:10258E00A3EDF0900033E0D39401401A90000AE0DE
:10259E00FEA3E0FFAC29AD2AEF2DFDEE3CFC900032
:1025AE000AECF0A3EDF0D219AE27AF2890000AE0A6
:1025BE00FCA3E0FDEFC39DEE9C40159000C7E0B478
:1025CE000104C2968002C2A07446900032F0C21975
:1025DE00A219B3B35007900032E0B53702801590C0
:1025EE0000C7E0B40104C2968002C2A074469000F7
:1025FE0032F0C219E54CB4020280030226B2124434
:10260E00B41245CB9007A9E0FEA3E0FF740A125165
:10261E003890000EE0FCA3E0FD74098F02FF12005B
:10262E00858D078C038E048A058B0612503A90070F
:10263E00ADEEF0A3EFF09000C7E0B401087450BE09
:10264E0000059F4002800D74509007ADF8E4F0E84D
:10265E00A3F0801B9007ADE0FEA3E0FF74F0BE0078
:10266E00039F500B74F09007ADF8E4F0E8A3F090E0
:10267E0007ADE0FEA3E0FFE55B2FFF50010E9007D4
:10268E00ADEEF0A3EFF0900048E0B40103754C0AF4
:10269E00900048E0B40203754C0B900048E0B40380
:1026AE0003754C0CE54CB401259000DEE09030CB68
:1026BE00F82828731242528012124252800D124292
:0B26CE00DC8008124388800312438860
:0F30CB000226C20226C70226CC0226D10226D632
:1026D900754C02A206B3401D75A710A207B3B350EB
:1026E90007E5CDC394BF40028004D2978002C29708
:1026F90075A700801B75A710A207B3B35007E5CDD6
:10270900C3944040028004D2978002C29775A70003
:10271900E54BC394094003022E54A2EDB3500302C2
:102729002E54C2EDE54B60030228C890007AE07090
:10273900030228B79000B0E0B40102800302281711
:1027490090003EE0B5370280030228147E017F0025
:10275900E5BE125138E5BD2FFF50010E8E338F347F
:1027690090007AE0B40118741012513890006FE0AB
:102779008E048F05FF120085ED900040F0802CAE8D
:1027890033AF34741012513890006FE08E048F0506
:10279900FF120085900040E02DFD50010C74018C62
:1027A900068D0712512AEF900040F0E54460089029
:1027B90000D6E06402600280219000D8E0B4011ADA
:1027C900900040E075F0E7A4FFAEF0E5448E048F79
:1027D90005FF120085ED900040F0900040E0FE906A
:1027E9000041E0D39E4004D21D8002B21D900040FA
:1027F900E0900041F09000ACE064016006A21DB3D6
:10280900B340028006900040E0F5380228B5D21D99
:102819007E017F00E5BE125138E5BD2FFF50010E44
:102829008E338F3490007AE0B40118741012513845
:1028390090006FE08E048F05FF120085ED90004037
:10284900F0802CAE33AF34741012513890006FE021
:102859008E048F05FF120085900040E02DFD500188
:102869000C74018C068D0712512AEF900040F0E597
:102879004460089000D6E06402600280219000D88C
:10288900E0B4011A900040E075F0E7A4FFAEF0E56E
:10289900448E048F05FF120085ED900040F09000F2
:1028A900ACE064016006900040E0F53880037538BB
:1028B90000900076E07005754B01800375BB18E543
:1028C9004BB401028003022A6A900076E070030289
:1028D9002A597E017F00E5BE125138E5BD2FFF5010
:1028E900010E8E338F349000BCE0B4010F7E0F7F50
:1028F900FFAC33AD341251978E338F349000E1E041
:10290900B40245AE33AF34900024E0FCA3E0FDED02
:10291900D39FEC9E400A900024E533F0A3E534F000
:10292900AE33AF34900026E0FCA3E0FDEFD39DEE7B
:102939009C400A900026E533F0A3E534F0AE33AFAE
:1029490034740412512A8F3A9000E1E0704CAE338E
:10295900AF34900024E0FCA3E0FDEFD39DEE9C4052
:10296900091251978E338F34800675340075330000
:10297900AE33AF34741012513890006CE08E048F6E
:1029890005FF1200858C338D347400D39D74019C2E
:10299900400585343A8003753AFF9000ACE0B401F4
:1029A900028003022A57A207B3B3500E900080E0B9
:1029B900A825B80005D395265003022A4C9000811A
:1029C900E075F019A4FFAEF09000C4E08E048F0505
:1029D900FF1200859000BDE0853AF0A4FFAEF074C7
:1029E900648D028C038E048F05FF120085EA2DFD8C
:1029F900EB3CFC8C338D34E544600F9000D6E0B499
:102A090002089000D8E0640160028017AE33AF3449
:102A190074E7125138E5448E048F05FF1200858C46
:102A2900338D34900040E0A833B8000AD395344080
:102A390005853438800BA21DB34006900040E0F5AF
:102A490038800BA21DB34006900040E0F5388003A2
:102A5900753A00900079E07005754B02800375BBEB
:102A690019E54BB402028003022B25900079E0702E
:102A790003022B14E537D3940C4003022B12900068
:102A890022E0FEA3E0FFE53E12518F900022EEF016
:102A9900A3EFF07E017F00E5BE125138E5BD2FFF9F
:102AA90050010E8E338F349000E6E07013740A12D1
:102AB900513874518E048F05FF1200858D3E80199F
:102AC900AE33AF34740A1251388F048E057E017FFC
:102AD90095CDCCCD12503A8F3EE53ED39464400358
:102AE900753E64900022E0FEA3E0FFE53E2FFF5013
:102AF900010E900022EEF0A3EFF090007DE0048E2D
:102B0900048F05FF1200858D3E8003753E329000CB
:102B1900C9E07005754B03800375BB13E54BB4031E
:102B29005E9000C9E060477E017F00E5BE12513822
:102B3900E5BD2FFF50010E8E338F34740412512AD4
:102B49008F3F9000CBE0853FF0A4FDACF07464FFAB
:102B59001200858D3F9000CAE0853FF0A4FFAEF0DA
:102B690074FF8E048F05FF1200858D4E8003753F1B
:102B790000900077E07005754B04800375BB17E57D
:102B89004BB404028003022C26900077E0B4017C48
:102B99007E017F00E5BE125138E5BD2FFF50010EC1
:102BA900740412512A8E338F34900043E0601290DE
:102BB9000043E014904F4893A833B8000695344079
:102BC900028006900043E014F0900043E0C394773C
:102BD9005013900043E004904F4893A833B8000580
:102BE900D3953450028006900043E004F0900043EE
:102BF900E0FE90009DE08E0088F0A4FFAEF07464C2
:102C09008E048F05FF1200858D408003754000906A
:102C19000078E07005754B05800375BB16E54BB46C
:102C290005028003022CB9900078E0B4017C7E0192
:102C39007F00E5BE125138E5BD2FFF50010E740427
:102C490012512A8E338F34900044E0601290004470
:102C5900E014904FC193A833B80006953440028020
:102C690006900044E014F0900044E0C394775013B8
:102C7900900044E004904FC193A833B80005D39560
:102C89003450028006900044E004F0900044E0FED5
:102C99009000A3E08E0088F0A4FFAEF074648E0467
:102CA9008F05FF1200858D41800375410075BB1F9B
:102CB900E54BB406337E017F00E5BE125138E5BD10
:102CC9002FFF50010E8E338F34740912513874E678
:102CD9008E048F05FF1200858D4390007FE07005FB
:102CE900754B07800375BB15E54BB40702800302DA
:102CF9002DFB90007FE07003022DEA7E017F00E545
:102D0900BE125138E5BD2FFF50010E8E338F34743A
:102D19000412512A8F4290007FE0B401159000D32C
:102D2900E08542F0A4FFAEF0740712512AEF900734
:102D3900B6F090007FE0B402159000D3E08542F030
:102D4900A4FFAEF0740712512AEF9007B5F0900076
:102D59007FE0B403028003022DE89000C0E0701CFC
:102D6900E542C3940A5002D201E542D39464400279
:102D7900C20190009FE090006AF0806390009FE09C
:102D890070349000D3E08542F0A4FFAEF074FF8E5A
:102D9900048F05FF120085ED90006AF0AE25AF267D
:102DA900741EBE0006D39F4002D201E53AD394E5D2
:102DB9004002C2018029E542C3940A500DAE25AFF5
:102DC90026741EBE0004D39F50028002D201E53A48
:102DD900D394E54002C20190009FE090006AF08020
:102DE900037542009000D6E07005754B08800375A5
:102DF900BB14E54BB408509000D6E060397E017FE2
:102E090000E5BE125138E5BD2FFF50010E8E338FFC
:102E190034EFD39421EE940E40057544FF8015AE2E
:102E290033AF34741012513874E38E048F05FF12D6
:102E390000858D44800375440090007AE060057533
:102E4900BB1A800375BB18054BD2ECAE27AF28EF30
:102E5900D39498EE943A50030230B9C20E753746AE
:102E69009000BBE070057549028003754903C29360
:102E7900C294C291C292C287C290E5B554EFF5B52A
:102E8900E5B554DFF5B5C296C295C2A0C297C2A2F4
:102E9900C2A1E5B5547FF5B5E5B554BFF5B5A21E98
:102EA900B34008E5B54404F5B58006E5B554FBF52E
:102EB900B5A210B3500EE53AD394334007E53AC3AF
:102EC90094CC4003022F6DE5B54401F5B574289003
:102ED9000068F0900075E075F064A4FFAEF08E35DF
:102EE9008F367402BE000AD39F40067536027535C7
:102EF9000075A71085F95085FA517E017F00E551CB
:102F0900125138E5502FFF50010E8E338F34AC35F6
:102F1900AD36EF2DFDEE3CFC8C358D36D293D29437
:102F2900D291E536F5FBE535F5FCE536F5E9E5350C
:102F3900F5EAE536F5EBE535F5EC9000B9E0B403D3
:102F49001ED292D287D290E536F5EDE535F5EEE55C
:102F590036F5FDE535F5FEE536F5CEE535F5CF7502
:102F6900A700D210E53AC3941A5002C21090000C7F
:102F790074FFF0A374DCF090009CE0900012F8E478
:102F8900F0E8A3F0C214C216C21874C8900028F061
:102F990074C890002CF074C8900030F0C211C212AD
:102FA900C213752600752500753C00C207756D00B2
:102FB90090001AE4F0A3F0754C1E9007ABE0FEA355
:102FC900E0FF7403125138740112512A9007A9EED7
:102FD900F0A3EFF090008EE060051248058002C270
:102FE90004900091E060051248F58002C206A2042F
:102FF900300501B35017A204B34008E5B54408F5FC
:10300900B58006E5B554F7F5B5A2049205C2037576
:103019002C00752B00900014E4F0A3F090007DE0E3
:1030290075F032A4FFAEF0900022EEF0A3EFF0901D
:103039000010E4F0A3F0C21F900070E4F0C209C2CE
:1030490008C21C900069E0C3943C5019758DA8759D
:103059008B00753D03E54BB40909900069E004F064
:10306900754B00803BE54BB40903754B007528008F
:10307900752700758D00758B00753D00900068E01F
:10308900C3943C5008900068E004F08006743C90BA
:103099000068F0900068E0B43C06E5B554FEF5B56B
:1030A900E543C394415009740E900045F01205F1AF
:0330B900020DC93C
:104ED0000000010001400160018001A001C001E06B
:104EE00002000300039603B603D603F40400050092
:104EF00005180530054805600578059005A805C02A
:104F0000060006140628063C066E068C00FF013FCC
:104F1000015F017F019F01BF01DF01FF02FF0395D8
:104F200003B503D503F303FF04FF0517052F05475A
:104F3000055F0577058F05A705BF05FF0613062743
:104F4000063B066F068B06A9DAD8D7D5D4D2D0CFC8
:104F5000CDCBC9C7C6C4C2C0BEBCBAB8B5B3B1AF69
:104F6000ADABA8A6A4A2A09D9B99969492908D8B80
:104F700089878482807E7C79777573716F6D6B69A8
:104F8000676563615F5D5B5957565452504F4D4B97
:104F90004A4847454442413F3E3C3B3A3937363523
:104FA000343231302F2E2D2C2B2A29282726252547
:104FB0002423222121201F1E1E1D1C1C1B1A1A190E
:104FC00019EEECEBEAE9E8E7E5E4E3E1E0DEDDDB5E
:104FD000D9D8D6D4D2D0CECCCAC8C6C3C1BFBCBA29
:104FE000B7B5B2B0ADABA8A5A3A09D9B9895929084
:104FF0008D8A8785827F7D7A7775726F6D6A686525
:1050000063615E5C5A575553514F4D4B4947454379
:1050100042403E3C3B393836353332312F2E2D2B32
:105020002A292827262524232221201F1E1D1D1C56
:0A5030001B1A1A1918181716161586
:1030DA00750B00750A00AE0AAF0BAC08AD09EDC35B
:1030EA009FEC9E401674FF12007575CF01780B7421
:1030FA000126F6500418E436F650DB2290003DE033
:10310A00B4AA1C900771E0B43C159007B1E0FEA385
:10311A00E0FFEF4E6009741EBE0004D39F50030205
:10312A00323475360075350075F8099007B1E0FE3E
:10313A00A3E0FF74076F4E6006740E6F4E7006743C
:10314A003A900771F09007B1E0FEA3E0FF7408BE61
:10315A00001ED39F401A7E017F089007B1E0FCA3AE
:10316A00E0FD1DBDFF011C1200038E338F34801F4A
:10317A009007B1E0FEA3E0FF740812518F8F048E0E
:10318A00057E017F08CDCCCD1200038E338F34AE7D
:10319A0035AF36740CD39F74019E500302322FA2AE
:1031AA00F9B3407EE5364535700375A382AE35AF77
:1031BA003674016F4E700375A300AE35AF367402D4
:1031CA006F4E700D9007B2E075F002A4FDACF08D61
:1031DA00A3AE35AF3674036F4E700375A300AE35D8
:1031EA00AF367403BE00039F5013AC33AD34ED2FDA
:1031FA00FFEC3EFE90006D12515FE0F5A3AE35AFD5
:10320A0036EFB40B09EEB401057414120075AE352D
:10321A00AF36EFB40B07EEB4010375F80D7835122B
:10322A00519F02319990003DE4F0227536007535C0
:10323A000075F8099007B1E0FEA3E0FF7408BE002C
:10324A001ED39F401A7E017F089007B1E0FCA3E0DD
:10325A00FD1DBDFF011C1200038E338F34801F90A9
:10326A0007B1E0FEA3E0FF740812518F8F048E05A8
:10327A007E017F08CDCCCD1200038E338F34AE355C
:10328A00AF367411D39F74019E5003023365A2F9BD
:10329A00B35003023362E5364535700375A3D2AEE7
:1032AA0035AF3674016F4E700375A300AE35AF3675
:1032BA0074026F4E700D9007B2E075F002A4FDAC77
:1032CA00F08DA3AE35AF3674036F4E700375A3004D
:1032DA00AE35AF3674046F4E700375A300AE35AFCA
:1032EA003674056F4E700375A300AE35AF3674069B
:1032FA006F4E700375A300AE35AF3674076F4E700C
:10330A000375A300AE35AF3674086F4E700375A30C
:10331A0000AE35AF367408BE00039F5016AC33AD0D
:10332A0034ED2FFFEC3EFE90006812515FE5A3F0EA
:10333A0075A300AE35AF36EFB41009EEB4010574CB
:10334A0014120075AE35AF36EFB41007EEB40103B0
:10335A0075F80D783512519F02328822753600753C
:10336A00350075F809AE35AF367417BE0004D39F21
:10337A00500302343EA2F9B3500302343BE536450A
:10338A0035700375A3D2AE35AF3674016F4E700334
:10339A0075A300AE35AF3674026F4E700D9007B24A
:1033AA00E075F002A4FDACF08DA3AE35AF36740320
:1033BA006F4E700375A300AE35AF3674046F4E704E
:1033CA000375A300AE35AF3674056F4E700375A34F
:1033DA0000AE35AF3674066F4E700375A300AE3576
:1033EA00AF3674076F4E700375A300AE35AF3674EF
:1033FA00086F4E700375A300AE35AF367408BE0071
:10340A00039F500C90005112515FE5A3F075A30081
:10341A00AE35AF3674166F4E70057414120075AE61
:10342A0035AF3674166F4E700375F80D7835125134
:10343A009F02336F2290003DE0B4AB028003023456
:10344A00D975360075350075F809AE35AF36741280
:10345A00BE007CD39F4078A2F9B34070E53645356B
:10346A00700375A382AE35AF3674016F4E70037563
:10347A00A300AE35AF3674026F4E700D9007B2E0FE
:10348A0075F002A4FDACF08DA3AE35AF3674036FB0
:10349A004E700375A300AE35AF367403BE00039FAA
:1034AA00500990005612515FE0F5A3AE35AF36745D
:1034BA00116F4E70057414120075AE35AF36741163
:1034CA006F4E700375F80D783512519F02345422ED
:1034DA00900046E4F074649007B1F8E4F0E8A3F0D1
:1034EA0012336674C89007B1F8E4F0E8A3F09000CC
:1034FA005DE0B4371A90005AE0900051F090005BFA
:10350A00E0900052F090005CE0900053F08046900A
:10351A0000467401F074659007B1F8E4F0E8A3F08E
:10352A0012336674C89007B1F8E4F0E8A3F090008B
:10353A005DE0B4371A90005AE0900051F090005BB9
:10354A00E0900052F090005CE0900053F080067426
:10355A0002900046F0900047E4F074669007B1F8D4
:10356A00E4F0E8A3F012336674C89007B1F8E4F007
:10357A00E8A3F090005CE0B4371290005AE09000A3
:10358A004BF090005BE0900054F080769000477416
:10359A0001F074679007B1F8E4F0E8A3F01233661B
:1035AA0074C89007B1F8E4F0E8A3F090005CE0B4C6
:1035BA00371290005AE090004BF090005BE09000C8
:1035CA0054F0803E7402900047F074689007B1F896
:1035DA00E4F0E8A3F012336674C89007B1F8E4F097
:1035EA00E8A3F090005CE0B4371290005AE0900033
:1035FA004BF090005BE0900054F08006740390005A
:10360A0047F022E55E2534FFAE3350010E9000717B
:10361A0012515FE0F55FE55E2534FFAE3350010ECF
:10362A000FBF00010E90007112515FE0F5608566D0
:10363A0062E55FB56005855F5E8041E560D3955FB1
:10364A00401DE560C3955F8561F0A4FFAEF0E562B9
:10365A008E048F05FF120085ED255FF55E801DE55E
:10366A005FC395608561F0A4FFAEF0E5628E048FBA
:10367A0005FF120085EDF404255FF55E22E560D3AF
:10368A00955F401DE560C3955F8561F0A4FFAEF0CC
:10369A00E5628E048F05FF120085ED255FF55E80D9
:1036AA001DE55FC395608561F0A4FFAEF0E5628E0B
:1036BA00048F05FF120085EDF404255FF55E22E50F
:1036CA003875F00484FF7E008F5EE53875F0048457
:1036DA00ADF07C008D61756604753301753400E5C3
:1036EA005EC3943F500512360D80069001B0E0F596
:1036FA005E855E54755300900042E075F020A4FF89
:10370A00AEF09000C2E08E048F05FF1200858D5E38
:10371A009000AAE0D3953850030237CF9000CEE04C
:10372A00D395384010ED9001B1125174E0F55675F9
:10373A0055000237CC900099E0D395384043E55EB6
:10374A009001B1125174E0F55FE55E9001D112511A
:10375A0074E0F5609000CEE0F4042538F56190003D
:10376A0099E0FE9000CEE0F4042EF562E55FB560C4
:10377A0005855F5E8003123687855E567555008023
:10378A0041E55E9001D1125174E0F55FE55E90016A
:10379A00F1125174E0F560900099E0F4042538F5CF
:1037AA00619000AAE0FE900099E0F4042EF562E52B
:1037BA005FB56005855F5E8003123687855E567544
:1037CA0055000238769000D1E0D395385011E55E65
:1037DA00900231125174E0F5567555000238769010
:1037EA00009AE0D395385043E55E90021112517465
:1037FA00E0F55FE55E900231125174E0F5609000E9
:10380A009AE0F4042538F5619000D1E0FE90009A20
:10381A00E0F4042EF562E55FB56005855F5E80031E
:10382A00123687855E567555008041E55E9001F136
:10383A00125174E0F55FE55E900211125174E0F5E1
:10384A00609000AAE0F4042538F56190009AE0FE41
:10385A009000AAE0F4042EF562E55FB56005855F85
:10386A005E8003123687855E56755500229000E207
:10387A00E0F563756611753302753400AE25AF261F
:10388A00E56375F00FA4FDACF0EDD39FEC9E4021EB
:10389A00E5638E048F05FF120085ED75F010A4FF15
:1038AA00AEF0E53875F01184FD7C00ED2FF56480EB
:1038BA000EE53875F01184FF7E00EF24F0F564857B
:1038CA00645EE53875F01184AFF07E008F611236C0
:1038DA000D855E65AE25AF269000E2E075F00FA477
:1038EA00FDACF0EDD39FEC9E402875330275341081
:1038FA0085645E12360D85655F855E60AE25AF26EE
:10390A00E5638E048F05FF1251538D618563621240
:10391A003687855E54755300755664755500229036
:10392A0000E2E0F563756611753302753400AE2561
:10393A00AF26E56375F00FA4FDACF0EDD39FEC9EC6
:10394A004021E5638E048F05FF120085ED75F010A6
:10395A00A4FFAEF0E53A75F01184FD7C00ED2FF579
:10396A0064800EE53A75F01184FF7E00EF24F0F5CD
:10397A006485645EE53A75F01184AFF07E008F616C
:10398A0012360D855E65AE25AF269000E2E075F031
:10399A000FA4FDACF0EDD39FEC9E40287533027561
:1039AA00341085645E12360D85655F855E60AE25CE
:1039BA00AF26E5638E048F05FF1251538D6185632F
:1039CA0062123687855E547553009000ACE0B404E9
:1039DA0053E53875F00484FF7E008F5EE53875F094
:1039EA000484ADF07C008D6175660475330175340D
:1039FA0000E55EC3943F500512360D80069001B073
:103A0A00E0F55EAE53AF54E55E12513874648E042D
:103A1A008F05FF120085AE53AF54EF2DFDEE3CFC2F
:103A2A008C538D5475566475550022900077E0B416
:103A3A000146E54075F00584FF7E008F5EE540751E
:103A4A00F00584ADF07C008D6175660575330575EA
:103A5A003400E55EC39417500512360D80069005B2
:103A6A0088E0F55EAE55AF56E55E2FFF50010E7445
:103A7A006412518F8E558F56900078E0B40146E556
:103A8A004175F00584FF7E008F5EE54175F005847F
:103A9A00ADF07C008D61756605753305753448E5B2
:103AAA005EC39417500512360D80069005D0E0F5D6
:103ABA005EAE55AF56E55E2FFF50010E746412518B
:103ACA008F8E558F56900087E0B40249E543C39420
:103ADA004175F00584FF7E008F5EE54375F005842D
:103AEA00ADF07C008D61756605753306753400E5A9
:103AFA005EC39413500512360D8006900684E0F5D5
:103B0A005EAE55AF56E55E2FFF50010E746412513A
:103B1A008F8E558F569000C9E0B402028003023B93
:103B2A00D4E53875F01584FF7E008F5EE53875F0B0
:103B3A001584ADF07C008D61756615753303753497
:103B4A00F4E55EC3940B500512360D80069004709E
:103B5A00E0F55EE55E75F0FFA4FFAEF09000CAE006
:103B6A008E048F05FF120085ED90006BF0E53F751E
:103B7A00F078A4FFAEF074FF8E048F05FF12008563
:103B8A008C338D3474028C068D0712512A8F5EACE9
:103B9A0033AD347404FF1251538D61756604753365
:103BAA000675346EE55EC3941D500512360D800607
:103BBA009006FCE0F55EAE55AF56E55E2FFF50016C
:103BCA000E746412518F8E558F562290007FE0B486
:103BDA0001179007B6E02556FFAE5550010E90002A
:103BEA00D3E012518F8E558F5690007FE0B40316A2
:103BFA00A201B3B3501090006AE0C39405A825B897
:103C0A0000069526400280109000A1E02556FFAEDE
:103C1A005550010E8E558F56900079E0B4020280FD
:103C2A0003023E0290007CE0602FE540D3941E40E0
:103C3A0028900014E0FEA3E0FF9000B7E075F003BF
:103C4A00A4FDACF0EFD39DEE9C400E9000DBE0A803
:103C5A0025B80005D395265003023E029000C4E021
:103C6A008538F0A4FFAEF07405125138740712516A
:103C7A002A8E338F34900083E0A825B80004952655
:103C8A005012900084E075F002A4FDACF0EFC39DE1
:103C9A00EE9C4003023E02E53875F00B84FF7E007D
:103CAA0090060112515FFEE0FFEE90007BE0FEEF0E
:103CBA008E0088F0A4FFAEF074648E048F05FF12A4
:103CCA0000858C338D34900042E075F018A4FFAE65
:103CDA00F09000C2E08E048F05FF1200858C068DDD
:103CEA000790061912515FAE33AF34E0125138749F
:103CFA00648E048F05FF1200858C338D34E53EA84F
:103D0A0033B80077D395344072E53EC39534FFE467
:103D1A009533FE8E338F347428BE00039F500C7582
:103D2A003428753300740D900045F0AE33AF3490EB
:103D3A00007CE012513874288E048F05FF1200852A
:103D4A008C338D34AE53AF54740A8E048F05FF1230
:103D5A0000858D068C07AC33AD34CFCECF1200036D
:103D6A00740A8E048F05FF1200858C338D34AE538E
:103D7A00AF541251978E538F54807DE53EA833B8C5
:103D8A00000495345072AE33AF34E53E12518F8E33
:103D9A00338F347428BE00039F500C753428753352
:103DAA0000740D900045F0AE33AF3490007CE01201
:103DBA00513874288E048F05FF1200858C338D3498
:103DCA00AE53AF54740A8E048F05FF1200858D0618
:103DDA008C07AC33AD34CFCECF120003740A8E04F5
:103DEA008F05FF1200858C338D34AE53AF54EF2DFF
:103DFA00FDEE3CFC8C538D5422AE53AF54AC55AD02
:103E0A005612000374648E048F05FF1200858C53CA
:103E1A008D54900074E08C068D0712513874648EAC
:103E2A00048F05FF1200858C538D54A2074017AEEC
:103E3A0025AF267405BE00039F5002D207E53AD388
:103E4A0094CC4002D2029000D6E0B402089000D886
:103E5A00E0640160028017AE53AF54E54412513852
:103E6A0074E78E048F05FF1200858C538D549000E1
:103E7A0096E05402601B90008DE0A825B80012D38A
:103E8A009526400DA207B3B35007E53AC3949A406A
:103E9A00028028AE5CAF5D90008BE075F002A4FD55
:103EAA00ACF0EF2DFDEE3CFC74022DFD50010CE54B
:103EBA003ABC0007D39D4003756A01853A5D755C7B
:103ECA0000E56A7003023F599000E9E0C3956A4031
:103EDA0070E54075F00584FF7E0090057112515F10
:103EEA00E0F534753300AE33AF3490009BE01251E5
:103EFA003874648E048F05FF1200858C358D3690D8
:103F0A0000E9E004C3956A8C068D071251389000C7
:103F1A00E9E08E048F05FF1200858C358D369000FE
:103F2A008CE08C068D07125138740A8E048F05FFB7
:103F3A00120085AE53AF54EF2DFDEE3CFC8C538D31
:103F4A0054056A9000E9E0C3956A5003756A0090C7
:103F5A000096E05401601B90008AE0A825B8001280
:103F6A00D39526400DA207B3B35007E538C394CCC6
:103F7A0040028025900088E075F003A4FFAEF0E5CA
:103F8A00672FFF50010E74032FFF50010EE538BE54
:103F9A000007D39F4003756B01853867E56B700393
:103FAA000240349000EAE0C3956B4070E54075F03A
:103FBA000584FF7E0090057112515FE0F534753378
:103FCA0000AE33AF3490009BE012513874648E0413
:103FDA008F05FF1200858C358D369000EAE004C308
:103FEA00956B8C068D071251389000EAE08E048F8B
:103FFA0005FF1200858C358D36900089E08C068D80
:10400A0007125138740A8E048F05FF120085AE53C9
:10401A00AF54EF2DFDEE3CFC8C538D54056B900094
:10402A00EAE0C3956B5003756B0090009BE0A853C0
:10403A00B800049554500990009BE0F5547553005C
:10404A00229000D7E0B401028003024156A207B3CE
:10405A0050030241549000A2E0B40168AE53AF5439
:10406A00AC25AD26120003743C8E048F05FF1200A6
:10407A00859000B2E0BC00109D400D9000B4E0A80D
:10408A0053B8000495545002D203AE53AF54AC2532
:10409A00AD26120003743C8E048F05FF1200859032
:1040AA0000B2E0C3940ABC0015D39D40119000B43D
:1040BA00E0C39405A853B80005D395545002800272
:1040CA00C2038068AE53AF54AC25AD261200037408
:1040DA00788E048F05FF1200859000B2E0BC0010B4
:1040EA009D400D9000B4E0A853B8000495545004C4
:1040FA00D2038038AE53AF54AC25AD2612000374F8
:10410A00788E048F05FF1200859000B2E0C3940AEE
:10411A00BC0015D39D40119000B4E0C39405A85388
:10412A00B80005D3955450028002C203A203B340DB
:10413A0019AE53AF549000B3E012513874648E0430
:10414A008F05FF1200858C538D548002C2039000A4
:10415A00D7E0B40258E53875F00884FF7E008F5E18
:10416A00E53875F00884ADF07C008D6175660875D8
:10417A0033017534E0E55EC3943F500512360D8075
:10418A0006900270E0F55EE55E75F05EA4FFAEF0A3
:10419A00740A8E048F05FF1200858C578D5874029D
:1041AA00BC000AD39D4006755802755700A200B399
:1041BA004006A202B3B3500990001AE4F0A3F080BB
:1041CA0024AE53AF547400D39F74019E400C9000E8
:1041DA001AE553F0A3E554F0800B74FF90001AF827
:1041EA00E4F0E8A3F09000B9E0D394024006A207F5
:1041FA00B3B34002800DAE53AF5474021251388EDD
:10420A00538F549000A2E0B4010DAE53AF54740220
:10421A001251388E538F54AE53AF54745E125138C4
:10422A00740A8E048F05FF1200858C538D54740214
:10423A00BC000AD39D4006755402755300900018BD
:10424A00E553F0A3E554F022900042E09003711286
:10425A005174E0F568756964900042E0FE9000AD23
:10426A00E0D39E4037E53875F00884FF7E008F5E04
:10427A00E53875F00884ADF07C008D6175660875C7
:10428A003303753496E55EC3941F500512360D80CC
:10429A0006900426E0F55E855E698035E53875F09E
:1042AA000884FF7E008F5EE53875F00884ADF07CE7
:1042BA00008D617566087533037534B6E55EC3947F
:1042CA001F500512360D8006900446E0F55E855EA5
:1042DA0069229000E3E0F56375661175330475345D
:1042EA0000AE25AF26E56375F00FA4FDACF0EDD363
:1042FA009FEC9E4021E5638E048F05FF120085ED39
:10430A0075F010A4FFAEF0E53875F01184FD7C005D
:10431A00ED2FF564800EE53875F01184FF7E00EF0D
:10432A0024F0F56485645EE53875F01184AFF07E9B
:10433A00008F6112360D855E65AE25AF269000E3CB
:10434A00E075F00FA4FDACF0EDD39FEC9E4028750C
:10435A00330475341085645E12360D85655F855E9B
:10436A0060AE25AF26E5638E048F05FF1251538D8B
:10437A0061856362123687855E687569642290007A
:10438A00E3E0F563756611753304753400AE25AF45
:10439A0026E56375F00FA4FDACF0EDD39FEC9E40CB
:1043AA0021E5638E048F05FF120085ED75F010A4D8
:1043BA00FFAEF0E53A75F01184FD7C00ED2FF5644F
:1043CA00800EE53A75F01184FF7E00EF24F0F56463
:1043DA0085645EE53A75F01184AFF07E008F611254
:1043EA00360D855E65AE25AF269000E3E075F00FC9
:1043FA00A4FDACF0EDD39FEC9E40287533047534D0
:10440A001085645E12360D85655F855E60AE25AFE8
:10441A0026E5638E048F05FF1251538D6185636211
:10442A00123687855E687569649000DEE0B40479A7
:10443A00900042E0FE9000ADE0D39E4037E538752B
:10444A00F00884FF7E008F5EE53875F00884ADF0D1
:10445A007C008D61756608753303753496E55EC315
:10446A00941F500512360D8006900426E0F55E85ED
:10447A005E698035E53875F00884FF7E008F5EE559
:10448A003875F00884ADF07C008D61756608753367
:10449A00037534B6E55EC3941F500512360D8006C7
:1044AA00900446E0F55E855E6922900077E0B401EB
:1044BA003BE54075F00584FF7E008F5EE54075F0B0
:1044CA000584ADF07C008D6175660575330575341C
:1044DA0018E55EC39417500512360D80069005A0A4
:1044EA00E0F55EE569255EC39464F569900078E0BD
:1044FA00B4013BE54175F00584FF7E008F5EE5411E
:10450A0075F00584ADF07C008D617566057533051F
:10451A00753460E55EC39417500512360D80069017
:10452A0005E8E0F55EE569255EC39464F569E5682A
:10453A002569F55B90007FE0B402109007B5E0258D
:10454A005BFE9000D3E0F4042EF55B9000D6E0D336
:10455A0094014040E544C394E7501D74E7C3954471
:10456A00FE9007B7E08E00F5F0E884FF7E008F5ECC
:10457A00E55B255EF55B801CE544C394E7FE900786
:10458A00B7E08E00F5F0E884FF7E008F5EE55BC33E
:10459A00955EF55BA2074006E5682464F55BE55B7A
:1045AA00D394644009E55BC39464F55B8003755B4F
:1045BA00009000AFE0C3955B50069000AFE0F55B5A
:1045CA0022D2009000C5E0A825B800049526503BE9
:1045DA009000C5E0A825B8000495265003755B0F26
:1045EA009000C5E004A825B8000495265003755B21
:1045FA000A9000C5E02402A825B8000495265005B3
:10460A00755B05C2007409900045F07E017F009039
:10461A0000B5E01251389000C4E08E048F05FF12F5
:10462A000085E538BC000CD39D4008C200740A908E
:10463A000045F09000B6E0C39540500D9000C8E0E8
:10464A00A825B80006952640028008C200740B907F
:10465A000045F0A2004003755B0590007FE0B403BB
:10466A0006A201B3B34002802B90006AE0C394050E
:10467A00A825B800049526500C9000A0E0F55B74BC
:10468A000C900045F090006AE0A825B80004952631
:10469A005002C200855B45900071E0255BFE9000E8
:1046AA0042E075F01E84FC7F00EE2CF55B22900040
:1046BA0042E075F00584FF7E008F5E900042E0754F
:1046CA00F00584ADF07C008D617566057533037560
:1046DA0034D69000C2E01475F00584FF7E00E55ED2
:1046EA00BE00039F500512360D800BE55E9004470D
:1046FA00125174E0F55EE55E9007B8F09007B8E0F5
:10470A00FE9000B1E0C39E50089000B1E09007B857
:10471A00F022E54075F00584FF7E00900571125184
:10472A005FE0F56DE56DD394644010E56DC3946464
:10473A0075F00F84FF7E008F6D8003756D00900009
:10474A0094E0256DF56D229007ABE0FEA3E0FF74BF
:10475A000412512AE538125138740F8E048F05FF5E
:10476A001200859007A9ECF0A3EDF0900087E0B461
:10477A000262E543C3944175F00584FF7E008F5EB3
:10478A00E54375F00584ADF07C008D6175660575AD
:10479A003306753414E55EC39417500512360D803E
:1047AA0006900698E0F55E9007A9E0FEA3E0FF7484
:1047BA000A8E048F05FF120085E55E8C068D0712AE
:1047CA005138740A8E048F05FF1200859007A9ECF0
:1047DA00F0A3EDF09007A9E0FEA3E0FF9007AFE099
:1047EA00FCA3E0FDEDD39FEC9E400F9007AFE0F8ED
:1047FA00A3E09007A9C8F0A3C8F02290008EE0B405
:10480A00010385265090008EE0B402129000C4E0A5
:10481A008538F0A4FFAEF0740812512A8F50900028
:10482A008EE0B40303853A5090008EE0B404038509
:10483A00405090008EE0B40507E541C39414F5504A
:10484A0090008EE0B4060385425090008EE0B407D3
:10485A000385435090008EE0B408038544509000CD
:10486A008EE0B40903853F5090008FE0FE900090DF
:10487A00E0D39E404B90008EE0B40418900090E084
:10488A00C395505002D20490008FE0D39550400255
:10489A00C204802A90008FE0C3955050099000907E
:1048AA00E0D3955050028002D20490008FE0D39555
:1048BA00505009900090E0C395505002C204802ADB
:1048CA0090008FE0D395504009900090E0C3955036
:1048DA0040028002C20490008FE0C39550400990C4
:1048EA000090E0D395504002D20422900091E0B4A7
:1048FA000103852650900091E0B402129000C4E0B2
:10490A008538F0A4FFAEF0740812512A8F50900037
:10491A0091E0B40303853A50900091E0B404038512
:10492A004050900091E0B40507E541C39414F55056
:10493A00900091E0B40603854250900091E0B407DC
:10494A0003854350900091E0B408038544509000D9
:10495A0091E0B40903853F50900092E0FE900093E5
:10496A00E0D39E4040900092E0C3955050099000D9
:10497A0093E0D3955050028002D206900092E0D381
:10498A0095505009900093E0C395505002C206908A
:10499A000091E0B401099000D0E0D3953A5002802A
:1049AA0002C206802A900092E0D3955040099000F6
:1049BA0093E0C3955040028002C206900092E0C381
:1049CA0095504009900093E0D395504002D20622B8
:1049DA00AE59AF5A74F5D39F74019E4008785912A4
:1049EA00519F024AD5755A01755900AE25AF26E581
:1049FA006DBE000DD39F40099000A6E0D3956E408E
:104A0A0002801B756E00E56DC39526F5509000A9CE
:104A1A00E0D3956C4006E56C2550F56C8002056E76
:104A2A00900082E0D3953A401CE538C39539401589
:104A3A00AE25AF26E56DBE00039F50099000A7E0A2
:104A4A00D3956F400280579007B9E0A825B80004B3
:104A5A00952650037571009007B9E0A825B8000B98
:104A6A00D395264006E5269007B9F0E571702AE548
:104A7A0026C3956DF550E550D3940540037550054E
:104A8A009000A8E0C3956C5007E550C3956C4002AE
:104A9A008007E56CC39550F56C756F008002056F51
:104AAA00E5717016900082E0C3953A500DE56D24C9
:104ABA0005A825B8000695264002800F900095E0CB
:104ACA00F56C75710174789007B9F022AE59AF5A36
:104ADA0074E9D39F74039E4008785912519F024C7F
:104AEA0083755A01755900756C32A220402A756C7B
:104AFA0019900095E075F002A4FFAEF0E56EBE00D5
:104B0A0006D39F4002D220056E7571037478900710
:104B1A00B9F0757000024C72AE25AF26E56D6F4E86
:104B2A007003024C72E56DBE000DD39F40099000E0
:104B3A00A6E0D3956E40028017756E00A207B3B344
:104B4A005007E571C3940340028003756C19800D08
:104B5A00E56DC39526F550E56E2550F56E900082F9
:104B6A00E0D3953A400E9007B9E0A825B80007D3DC
:104B7A0095264002800C0570900095E0B57003758B
:104B8A007100E571B4030DE56D2402A825B800068D
:104B9A0095264002800A0570E570B43C03757102DF
:104BAA00E571B402299007B9E0A825B8000ED3959B
:104BBA00264009E5269007B9F0757000900082E05A
:104BCA00C3953A500975700074789007B9F0E57189
:104BDA00705A900082E0D3953A401CE538D3953953
:104BEA004015AE25AF26E56DBE00039F5009900023
:104BFA00A7E0D3956F40028008756F00756C4B80F3
:104C0A0028E526C3956DF550E550D3940540037504
:104C1A005005900082E0D3953A4008E56F2550F59B
:104C2A006F8006E56F2406F56F757000E5717016E2
:104C3A00900082E0C3953A500DE56D2405A825B889
:104C4A000006952640028003757101E571B40118CA
:104C5A00756C190570900095E0B57006757102754E
:104C6A00700074789007B9F0E56C75F00AA4FFAE8D
:0A4C7A00F09007B3EEF0A3EFF02274
:095174002582F582500205832218
:0F511B0025E050020583258250020583F582228C
:10006400EF2F500205832582F582E5833E2EF5832A
:010074002269
:10518F00CFC39FFF50011E22C3EF9DFFEE9CFE2257
:09517D00E493F608740193F62294
:08519F000806B6000218062202
:0D514600A3E004F0700612516AE004F022AC
:0E003900A3E014F0B4FF0612516AE014F022A6
:0E512A00048007C3CE13CECF13CFD5E0F622FC
:10503A00BC000FBE0008ED8FF084FFADF022E4FE45
:10504A00FF22BE000DEF60FE54F0606F20E70302FE
:10505A0050F0EAC0E0EBC0E078017A0075F001EEAA
:10506A0020E710EF25E0FFEE33FE0AC5F023C5F076
:10507A0030E7F0EA5407F9096A7A007B0060010810
:10508A00C3EC9E40167004ED9F4010ED9FFDEC9E10
:10509A00FCE5F0CA4ACA03F5F08005E5F003F5F02D
:1050AA00C3EE13FEEF13FFD9D77908CACBCAD8D0FB
:1050BA00EAFEEBFFD0E0FBD0E0FA22EC8FF084FCB2
:1050CA00ED54F045F0C48FF084FEEDC454F045F081
:1050DA00C48FF084FDEEC4FE54F02DFFEE540F3C55
:1050EA00FEADF07C0022790078008FF0EC7E08207B
:1050FA00E70DC3CD33CD33C933C9C833C8DEF08415
:10510A0049F9E5F08FF0BE00E6FD7C00E9FFE8FE14
:01511A002272
:0E513800F88FF0A4FFE5F0CE88F0A42EFE2242
:10000300EF8DF0A4F9A8F0EF8CF0A428F8EE8DF0B2
:06001300A428FEE9FF2213
:10007500600D782B02007F007830D8FED5E0F8229D
:10008500EEC0E07E0012503AEFFDEEFCD0E0FE221D
:0C515300EEC0E07E0012503AD0E0FE22D8
:03001B0002001EC2
:03009B0002004917
:0300000002518624
:0951860075817275D00002072F3B
:10515F00E5822FF582E5833EF583220582D5820213
:05516F001583158222EA
:10001E00C0E0C0F0C083C082C0D075D0001206C947
:0B002E00D0D0D082D083D0F0D0E032E0
:10004900C0E0C0F0C083C082C0D075D0001206CC19
:0B005900D0D0D082D083D0F0D0E032B5
:00000001FF
